:100000000C949C030C94B9030C94B9030C94B9039D
:100010000C94B9030C94B9030C94B9030C94B90370
:100020000C94B9030C94B9030C94E6180C9428189A
:100030000C9487210C94B9030C94B9030C94B90364
:100040000C94B9030C94B9030C94B9030C94B90340
:100050000C94B9030C9446210C94B9030C94B90385
:100060000C94B9030C94B9030C94B9030C94B90320
:100070000C94B9030C94B9030C94B9030C94B90310
:100080000C94B9030C94B9030C94B9030C94B90300
:100090000C94B9030C94B9030C94B9030C94B903F0
:1000A0000C94B9030C94B9030C94B90376067C063E
:1000B0006A067006820688068E060E070E073D0742
:1000C0003D07B807D607D808D808DB074F086008EF
:1000D0006008970606090B09100915091A091F0976
:1000E000240929092E0933096B043A093D094009FD
:1000F0004309460949094B094E0950093B16621646
:10010000101862161018AE16D1161018C617D6178A
:100110008E1C931C9D1C911C961C9B1C991C301EB4
:10012000331E361E391E3C1E3F1E421E00000000BC
:1001300000000000000000000000000000000000BF
:1001400000000000000000000000000000000000AF
:100150007E0F00D4FFFFFFC7000000780000000002
:10016000000000002A2B2800000000000000000012
:100170000000000000000029000000002C1E3420B8
:10018000212224342627252E362D3738271E1F20DE
:100190002122232425263333362E37381F04050623
:1001A0000708090A0B0C0D0E0F1011121314151667
:1001B0001718191A1B1C1D2F3130232D3504050665
:1001C0000708090A0B0C0D0E0F1011121314151647
:1001D0001718191A1B1C1D2F3130354C1E0F050026
:1001E000047F3F1F643214643214783C1E1E140ACC
:1001F0000529002B0029211A7CA90000001E0014EB
:100200000004001D00AA00E2001F001A0016001BD7
:1002100000BD00E3002000080007000600BE002C1F
:1002200000210015000900190028784D0022001750
:10023000000A0005000000C15200572D0000002FE9
:100240000000004A00A8002E000000300000004B13
:100250000023001C000B00110000003500240018D2
:10026000000D00100027784E0025000C000E00360F
:1002700000037E2822260012000F003700047E2A89
:100280000027001300330038000157C152350031F8
:100290000034001B7CC15200002900010001000154
:1002A00000010000003A00D100CF000100010072FF
:1002B0007C3B00CD00CE00D300010001003C00D209
:1002C00000D0000100010001003D00D900DA00016A
:1002D00000010001003E00010035000100000001A6
:1002E0000044000100000001000000010045000181
:1002F0000000000100000001003F0001005000016B
:100300000000000100400001005100010001000157
:100310000041004900520001000100010042004676
:10032000004F00010001004C0043000100010001EA
:1003300000010001000100010001000100010000B6
:100340000005010980A101850319012AB7001501E3
:1003500026B700950175108100C0050C0901A101A7
:10036000850419012AA002150126A0029501751025
:100370008100C005010906A1018506050719E029CC
:10038000E715002501950875018102050719002967
:10039000EF1500250195F075018102050819012965
:1003A00005950575019102950175039101C005013F
:1003B0000902A1010901A100050919012908150077
:1003C0002501950875018102050109300931158162
:1003D000257F95027508810609381581257F9501CD
:1003E00075088106050C0A38021581257F9501756F
:1003F000088106C0C00660FF0961A10109621500FD
:1004000026FF009520750881020963150026FF006C
:10041000952075089102C005010906A1010507197B
:10042000E029E71500250195087501810295017500
:100430000881010507190029FF150026FF00950610
:100440007508810005081901290515002501950584
:1004500075019102950175039101C00902740004B0
:100460000100A0FA090400000103010100092111A3
:10047000010001224400070581030800010904016D
:1004800000020300000009211101000122220007DF
:10049000058303200001070504032000010904026D
:1004A0000001030102000921110100012247000798
:1004B000058203080001090403000103000000098C
:1004C0002111010001226D000705850320000112A2
:1004D0000100020000000897327549010001020086
:1004E0000122034500720067006F0044006F00782E
:1004F00000200045005A0020005300680069006E8B
:10050000006500000028035A0053004100200054F9
:10051000006500630068006E006F006C006F00678C
:1005200000790020004C00610062007300000004AC
:100530000309042223252628292A2C2D2F30323383
:100540003536383A3B3D3E4042434547494A4C4E9A
:100550005051535557595A5C5E6062646668696BC6
:100560006D6F71737577797B7D7F81838587898ACC
:100570008C8E90929496989A9C9E9FA1A3A5A7A8D2
:10058000AAACAEAFB1B3B4B6B8B9BBBCBEBFC1C202
:10059000C3C5C6C7C9CACBCCCDCED0D1D2D2D3D495
:1005A000D5D6D7D7D8D9D9DADADBDBDBDCDCDCDCB3
:1005B000DCDDDDDDDDDCDCDCDCDCDBDBDBDADAD981
:1005C000D9D8D7D7D6D5D4D3D2D2D1D0CECDCCCB03
:1005D000CAC9C7C6C5C3C2C1BFBEBCBBB9B8B6B421
:1005E000B3B1AFAEACAAA8A7A5A3A19F9E9C9A98B1
:1005F000969492908E8C8A89878583817F7D7B7982
:10060000777573716F6D6B6968666462605E5C5A62
:100610005957555351504E4C4A4947454342403E25
:100620003D3B3A3836353332302F2D2C2A292826B7
:100630002523220001010101010101010102020241
:10064000020202020202030303030303030304047E
:100650000404040404050505050506060606060748
:100660000707070708080808090909090A0A0A0B01
:100670000B0B0C0C0C0D0D0D0E0E0E0F0F0F1010A2
:100680001111111212131314141515161617171829
:100690001819191A1A1B1B1C1D1D1E1E1F20202194
:1006A0002222232424252626272829292A2B2C2DDB
:1006B0002D2E2F30313232333435363738393A3BFC
:1006C0003C3D3E3F404142434445464748494A4CF1
:1006D0004D4E4F50515354555658595A5B5D5E5FBD
:1006E000616264656668696B6C6D6F707273757753
:1006F000787A7B7D7E8082838587888A8C8E8F91B5
:10070000939596989A9C9EA0A2A3A5A7A9ABADAFDE
:10071000B1B3B5B7BABCBEC0C2C4C6C9CBCDCFD1C8
:10072000D4D6D8DBDDDFE2E4E7E9EBEEF0F3F5F871
:10073000FAFDFFFFAA7F554011241FBECFEFDAE07C
:10074000DEBFCDBF11E0A0E0B1E0E6E6FCE502C00F
:1007500005900D92AC3CB107D9F723E0ACECB1E0C9
:1007600001C01D92A03BB207E1F70E945A090C9408
:10077000312E0C940000A0E0B0E0E1ECF3E00C942A
:10078000302BFC012481222309F48FC57C0161E018
:100790000E948B1BEC01F7018581882309F42AC58F
:1007A0008091690390916A03009709F45EC0C817AD
:1007B000D90709F45AC0992764E0880F991F6A95F0
:1007C000E1F7FC01E75EFE4F2081246020838C5E10
:1007D0009E4FFC01D183C0830E9483221092680344
:1007E00061E0C7010E948B1BEC0181159E4709F057
:1007F00040C0F7018581882309F401C59091D90192
:1008000081E0890F8770987F853020F4892B809351
:10081000D90102C09093D9018091D9018770FFEF6F
:100820008F9FC00111249595879595958795992758
:10083000909389008093880090938B0080938A0026
:1008400090938D0080938C004091D9015091DA01F2
:100850006091DB017091DC018FE090E00E94F72B4A
:100860008091EC010E946E1CCAC4C115FEE7DF072F
:1008700029F2F7018581C230FEE7DF07F1F028F4A5
:10088000C1303EE7D307E9F02FC0C3304EE7D407AD
:1008900029F0C4305EE7D50731F026C0882341F047
:1008A0008FE992E007C0882319F081E292E002C04C
:1008B00080E090E00E940D2240C2882309F43DC2EE
:1008C0000AC0882309F439C29091CE0181E08927BA
:1008D0008093CE0132C281E004C0816080935D03C9
:1008E00086950E94912629C29E0137552F3F3105DA
:1008F00011F008F059C06E01DD24960144E0220F8A
:10090000331F4A95E1F789010C5E1E4FF901E75E3E
:10091000FE4F6F01908180FB90F99083F7018581F4
:10092000882341F10E947B2190930D0280930C0259
:10093000F80182818F5F82839091680380919E028B
:10094000892B8383809191028483468157816685B8
:100950007785C8010E946422F601808181FF03C06F
:1009600090E080E002C09C2F8D2F909369038093CC
:100970006A031AC0F8014485558566857785C801E4
:100980000E946422F601808181FF0EC0C8010E948E
:100990006A228091690390916A038C179D0721F464
:1009A00010926A0310926903F7018581882309F484
:1009B0000DC1C137FCE7DF0709F4F8C0C2372CE7E7
:1009C000D20709F4F9C0C0373CE7D30709F0FEC0ED
:1009D000809038019090390180910A0190910B012B
:1009E0008816990639F48091D501803219F48FEC7C
:1009F00091E037C090920B0180920A0180E28093CF
:100A0000D501A12CB12C1092D40104ED11E0C0E06D
:100A1000D0E02AE0422E512C612C712CC501B4018A
:100A2000A30192010E944B2C605D603311F420976A
:100A300039F081149104A104B10419F460E201C0F9
:100A400060E3F80162938F01C501B401A301920133
:100A50000E944B2C49015A012196C530D105F1F66F
:100A6000C6CFEC01019628812032D9F39AE0892E75
:100A70002881222309F461C1213009F041C0898114
:100A8000813039F48E010E5F1F4F8A810E942B2A1C
:100A900008C0823041F48E010E5F1F4F8A810E9490
:100AA0006829E80181C0833039F48E010E5F1F4F41
:100AB0008A810E940429F5CF843011F0219674C0F8
:100AC0002A81229680E090E030E0205331092A30DC
:100AD000310558F4889EA001899E500D1124C9014A
:100AE000840F951F21962881EFCF009709F45CC0F1
:100AF000EFE9FFE03197F1F700C000000197F5CF73
:100B0000E22FF0E0E45AFE4F9490822F869586956E
:100B1000869590E0FC01E45BFE4FC4902770D12CD9
:100B2000022E02C0D594C7940A94E2F7F1E0CF22D6
:100B3000DD24FC01E45CFE4FA490B12C022E02C027
:100B4000B594A7940A94E2F731E0A322BB24FC01F8
:100B5000E45DFE4F049110E002C0159507952A95BB
:100B6000E2F701701127C114D10419F081EE0E943F
:100B70006829A114B10419F086EE0E946829892D14
:100B80000E942B2AA114B10419F086EE0E940429B8
:100B9000C114D10419F081EE0E9404290115110538
:100BA00019F08CE20E942B2A219662CF80913801A5
:100BB00090913901059605C08091380190913901D5
:100BC00005979093390180933801B7C0AE01FE01BB
:100BD000E851FC47E730F10508F478C0882309F4B0
:100BE000BEC010926703C3304CE7D40709F459C064
:100BF00048F4C1158CE7D807A9F0C130DC4709F4E7
:100C000056C0B7C0CB35ECE7DE0709F45BC0CC3586
:100C1000FCE7DF0709F44EC0CA35DC4709F0A9C07C
:100C200081E051C010929E020E94DD273FEF44E315
:100C30005CE0315040405040E1F700C00000F894C3
:100C400081E08093E00080E28093D8001092C90098
:100C50008FE19EE40197F1F700C000001DBA1092E9
:100C600068001CBC10BE1FBA10927A0010926E0071
:100C700010926F0010927100109272001092C900D1
:100C80001092BC0014B817B81AB81DB810BA109258
:100C9000BC0015B818B81BB81EB811BA0C94003FA8
:100CA0004CC06FEF7FEF80E090E00E94032C0E9429
:100CB000561C43C080919C0282FB882780F991E0FA
:100CC000892701C080E00E94591153C0EA5AFF4FA2
:100CD0000C94AA2C06E221EE41EE6AE17CE723C0E7
:100CE00007E225EE45EE6BE17CE71DC006E221EE52
:100CF00040EE68E17CE717C007E225EE44EE69E1CB
:100D00007CE711C006E221EE42EE6CE17CE70BC00D
:100D100007E225EE46EE6DE17CE705C008E221E042
:100D200045EE6EE17CE7C7010E94AD2206C08091CE
:100D30005D0380FFD2CD0E9456248091700287709F
:100D400009F4B3C2F7018581882309F4AEC280910A
:100D50009C0282FFAAC282E00E944211A6C2809138
:100D60009E028272FA01E052F847E531F10508F47B
:100D700049C2F7018581C081D181882349F0CE0124
:100D80000E94D126182F682FCE010E94412704C04F
:100D9000CE010E940D27182FBE01812F0E94290F1E
:100DA0000E94460FD82FC92FC82EF7011581068142
:100DB00002950F7080917002877001F11123F1F09C
:100DC000892F807F803469F080E28D0F8830B0F009
:100DD000892F807E803229F4F1E0FD1778F400231A
:100DE00069F080919C0282FF09C082E00E9442115A
:100DF000809170028770DD24D3948111D12CBC2E98
:100E0000B2948FE0B8228B2D90E08C30910508F0E1
:100E1000CFC1FC01E35AFF4F0C94AA2C8C2F807F8A
:100E2000CF70882311F0C295C07F1123B9F0CC2375
:100E300009F4ACC180E28D0F883010F0C11006C0FB
:100E400090919E02C92BC0939E0205C090916803A9
:100E5000C92BC09368030E94ED1098C18D2F0E948A
:100E60000429CC2309F4A4C1D05E8C2FD83068F1BA
:100E7000CC2059F10E94DF102AC08C2F807FCF70C8
:100E8000803211F0C295C07FCC2029F021E0C2163B
:100E900009F44CC054C080919C0282FD1BC01123F8
:100EA00069F0CC2339F090919E02C92BC0939E0229
:100EB0000E94ED1080E00E9468297AC180E00E94C3
:100EC0000429CC2309F474C18C2F0E94E6100E94DF
:100ED000ED106EC1112381F00023A9F1013009F05A
:100EE00067C1909191028C2F8923C81709F460C1C2
:100EF000C92BC09391025CC101115AC18C2F0E9471
:100F00001B28809191029C2F982329F09C2F90956B
:100F10008923809391028091D6019C2F982309F414
:100F200047C1C0958C238093D60142C1112321F083
:100F3000023008F03DC107C001113AC115C01123AC
:100F400031F0011123C18C2F0E94222831C10023CE
:100F500059F0D93309F029C13FEF47EE53E0315042
:100F600040405040E1F71FC18C2F0E941B2820C138
:100F70008C2F86958695837019F0813061F018C1A9
:100F8000112321F08D2F9C2F937002C080E090E000
:100F90000E94322213C1112321F08D2F9C2F9370B8
:100FA00002C080E090E00E940D2208C1612F8D2FC9
:100FB0000E942C2803C18C2F8370A9F51111FCC04D
:100FC0004D2F429546954770440F440F8D2F8F70DB
:100FD00090E09C01042E01C0220F0A94EAF7D4FF8E
:100FE00008C08FE090E001C0880F4A95EAF780952D
:100FF00001C080E0C695C695C370C23069F088F420
:1010000090919202C13019F0822B892302C0922B59
:10101000892B0E94B727D0C0822B909192028927FA
:10102000F8CF822BF6CF112319F08C2F817001C0DD
:101030008695882309F4C0C04D2F42954695477088
:10104000440F440F8D2F8F7090E09C01042E01C03F
:10105000220F0A94EAF7D4FF08C08FE090E001C0A5
:10106000880F4A95EAF7809501C080E0C695C6953D
:10107000C370C23059F078F49091EC01C13019F08E
:10108000822B892309C0922B892B06C0822B909139
:10109000EC01892701C0822B0E9476278DC0CF707A
:1010A000112339F08C2F0E94AB278D2F0E9422280C
:1010B00083C08D2F0E941B288C2F0E949E277CC0EE
:1010C0008D2F92EFC91661F19C1538F0E0EFCE1626
:1010D00059F0F1EFCF16F9F055C023EFC21639F1F0
:1010E00034EFC316A1F04EC0112369F0011160C0A6
:1010F000CF7181E090E001C0880FCA95EAF7909126
:10110000EC0189271EC0023008F052C0F1CF809157
:101110009C0282FD19C0112329F08C2F8F7126C0EB
:101120001123D9F38C2F8F710E949E2741C0112368
:1011300039F0CF7181E001C0880FCA95EAF701C08C
:1011400080E00E94762734C0112399F0CF718C2F54
:101150000E94AB2780919C0282FF07C048E0C49F99
:10116000C00111248360809370028C2F0E94AB27F2
:101170001FC081E00E9442110230D0F082E00E9444
:10118000421116C0112321F0002339F28D2F93CE86
:10119000002341F2893349F45FEF87EE93E0515029
:1011A00080409040E1F700C000008D2F0E9404298C
:1011B00088EF8B0D843010F40E945722DD20A9F0B7
:1011C0008091700280FD11C0F70115828695869589
:1011D00086950E94AB27C7010E94BB0380917002D5
:1011E0008695869586950E949E2760E0C7010E949D
:1011F0008B1B5BC0C1152EE7D20709F03ACBC0E0CC
:10120000DEE7D2CBE759FF4F0C94AA2C45E956E212
:101210006FE976E22CC04FE956E265E976E227C035
:1012200043ED55E26DED75E222C04DED55E263ED03
:1012300075E21DC049EB55E266EC75E218C046EC5C
:1012400055E269EB75E213C04FE955E26CEA75E2CD
:101250000EC04CEA55E26FE975E209C042E254E281
:101260006CE374E204C04CE354E262E274E20E9474
:101270003E2363CD65E082E015C068E086E012C0E1
:101280006EE089E00FC064E18FE00CC067E185E1AA
:1012900009C088E126CB62E289E104C083E221CB68
:1012A0006AE285E20E942B2348CDCDB7DEB7E0E1AC
:1012B0000C944C2BA6E4B0E0E0E6F9E00C94322B61
:1012C00085B7806885BF85B7806885BF84B7877F0D
:1012D00084BF0FB6F894A8958091600088618093D0
:1012E0006000109260000FBE90E080E80FB6F894A6
:1012F00080936100909361000FBE8CE19EE090931B
:10130000CD018093CC010E946C180E948B188091B3
:10131000E20084608093E20078948091CE0288237A
:10132000A1F01091E9001F709091EC00892F81705D
:1013300090FD80E8182B1092E9008091E80083FD71
:101340000E9456151F701093E90082E084BD93E05F
:1013500095BD9AEF97BD80936E000E940B1D90E0A3
:1013600090933C0180933B010E94461E0E948C1E7C
:10137000EDEDF1E0AFEEB1E011921D9221E0EB3E18
:10138000F207D1F78EE090E00E94F62C8093D7010F
:101390009093D801FC010E9611928E179F07E1F7EA
:1013A00089EA8093800089E08093810024982C98BA
:1013B0003F988AB18F7C8AB96E98479A8BB18063C7
:1013C0008BB9769A8FE090E00E94C92B6093D90187
:1013D0007093DA018093DB019093DC0167708FEFEB
:1013E000689FB00111247595679575956795772766
:1013F000709389006093880070938B0060938A00DB
:1014000070938D0060938C000E94821D80E090E0BC
:101410000E94CF2B863E9E4F11F00E94631082E007
:1014200090E00E94C12B8093FD0184E090E00E9437
:10143000CF2B90939C0280939B0283E090E00E94CC
:10144000C12B0E94B7278091EC010E946E1C8091F5
:10145000EB01811176C080E090E00E94CF2B863EA8
:101460009E4F21F00E9463100E94692488E090E062
:101470000E94C92B4B015C0184E290E00E94C12BC9
:10148000282F30E040E050E060E070E080E090E045
:1014900000E20E94BF2C282939294A295B29209380
:1014A0005D0330935E0340935F035093600360934A
:1014B00061037093620380936303909364032E7FB0
:1014C00089F50E94692488E090E00E94C92B6B0195
:1014D0007C0184E290E00E94C12B282F30E040E0A4
:1014E00050E060E070E080E090E00E94BF2CB22FFE
:1014F000A32FF42FE52F5B0197018601BC29A12BB7
:10150000F22BE32BB0935D03A0935E03F0935F0394
:10151000E093600360936103B0926203809363037E
:10152000909364030E94E92310928A0380915D03E3
:1015300080FF04C060E086950E944E2681E0809383
:10154000EB018091EC010E946E1C8CE091E0909385
:101550006E0380936D0388E1E82EF12C8091CE021A
:10156000853009F07EC000E4D02ECC24C39400E185
:1015700012E18091CE02853009F05CC08091CE02EC
:10158000843009F434C010928A038091EE018111F5
:101590000DC0C092EE0180915D03982F91709093E1
:1015A000ED018E7F80935D030E94452310927103AD
:1015B0000FB6F894A895E09260000FBED09260003C
:1015C00083B7817F846083BF83B7816083BF789452
:1015D000889583B78E7F83BF0FB6F894A8958091C6
:1015E0006000886180936000109260000FBE80915F
:1015F000C202882309F4BDCF0E940B1D90E0909396
:101600003C0180933B010E94461E0E948C1EEFEE1F
:10161000F1E0119221E0ED3FF207D9F70E94721339
:10162000EFEEF1E081918111E6C281E0ED3FF80734
:10163000C9F79FCF10929E020E94DD270E94572279
:101640001092EE018091ED01882349F080915D03B5
:10165000816080935D0360E086950E944E260E9423
:1016600038260E9472131EEFC12E11E0D12E2CE0FD
:1016700032E0AFEEB1E0F60191918D9189272E17FE
:101680003F0719F08823C1F305C0811103C00E94F0
:101690004E1454C0BFEE8B2EB1E09B2E10E0F4012F
:1016A00071904F01F601A080A724B1F100E0BB24A6
:1016B000B394662463948A2D8B2141F122960FAF57
:1016C000229723961FAF23970E947B2125969FAFD9
:1016D0008EAF259726966FAE269791E0872D8B21AA
:1016E00009F490E027969FAF279722964FAD229757
:1016F00023965FAD239724966FAD249725967FADF3
:10170000259726968FAD26970E94B61B0F5FBB0CC0
:10171000063089F6F60170821F5FFFEFCF1ADF0AED
:101720001E3009F0BCCF8FB7F894409172035091EE
:10173000730360917403709175038FBF8091690387
:1017400090916A03892B09F180910C0290910D020E
:101750000E946C21209138013091390128173907F6
:10176000A0F48091690390916A039927A4E0880FFF
:10177000991FAA95E1F7FC01E75EFE4F208122FD4B
:1017800004C08C5E9E4F0E94832280918A0388232E
:1017900009F4A5C080918903E0915D03E695E81BFB
:1017A000E0938503823059F4F0E0E351FE4FE49179
:1017B0000E2F10E0FEE0CF2EF1E2DF2E6BC0863060
:1017C00059F4F0E0E651FE4FE4910E2F10E0EEEFF9
:1017D000CE2EE0E2DE2E5EC0893061F4E695F0E0C8
:1017E000E951FE4FE4910E2F10E07AE9C72E70E226
:1017F000D72E50C08F3061F4E695F0E0EC51FE4FEB
:10180000E4910E2F10E064E3C62E60E2D62E42C0B3
:10181000853159F4F0E0EF51FE4FE4910E2F10E0C6
:1018200054EEC52E5FE1D52E35C08831F9F08332F4
:1018300049F4EFEDF1E00591149144ECC42E40E23F
:10184000D42E28C08432C9F08532F1F48E2F63E0A3
:101850000E947C2CE92FF0E0E452FE4FE4910E2F21
:1018600010E03DE9C32E3EE1D32E14C008E210E0A3
:1018700029E6C22E2FE1D22E0DC004EF11E091E334
:10188000C92E9FE1D92E06C000ED17E08CE9C82EC5
:101890008EE1D82E80918603882361F01092860312
:1018A0000E947B219093840380938303109288038A
:1018B000109287030E947B21E0918303F0918403BF
:1018C0008E1B9F0B8F3F9F4750F40E0F1F1F1093CF
:1018D00084030093830383E893E0F6010995B090B5
:1018E0007D03C0907E0310917F03D0908003009110
:1018F000810310927E0310927F0310928003109256
:101900008103C11003C0112309F447C080917B03F8
:1019100090917C030E946C219C0190917603992305
:1019200009F481C125313105C0F19F3F19F09F5F56
:1019300090937603CC2061F00E9407261C1414F4C7
:1019400091E001C09FEF899F802D112480937E0339
:10195000112361F00E940726111614F09FEF01C0B9
:1019600091E0899F802D112480937F0380917E03D5
:10197000882399F0A0907F03AA2079F00E942A265C
:10198000811101C081E080937E038A2D0E942A2666
:10199000811101C081E080937F03D11003C0002337
:1019A00009F447C08091790390917A030E946C21D9
:1019B0009C0190917703992309F439C125313105B0
:1019C000C0F19F3F19F09F5F90937703DD2061F096
:1019D0000E94E7251D1414F491E001C09FEF899F38
:1019E000802D112480938003002361F00E94E7255D
:1019F000101614F09FEF01C091E0899F802D1124F3
:101A00008093810380918003882399F0A0908103C3
:101A1000AA2079F00E942A26811101C081E08093DA
:101A200080038A2D0E942A26811101C081E08093C3
:101A3000810380917D038B111AC080917E038823DE
:101A400011F08C1114C080917F03882311F01813BA
:101A50000EC080918103882311F0081308C0909173
:101A60008003992331F081E0D91204C002C081E0E3
:101A700001C080E080FD15C080917E0381110FC000
:101A800080917F0381110BC080918003811107C079
:101A900081E090918103911103C080E001C081E059
:101AA00080FD0E94AA26B0927D03C0927E0310930F
:101AB0007F03D0928003009381030E94572290916C
:101AC0000E02891769F080930E028FB7F894409147
:101AD00072035091730360917403709175038FBF0B
:101AE0008091CE02843009F039CD8093E900809155
:101AF000E80082FF33CD8091E80085FF22C00E947C
:101B0000BD1981111CC000E210E06E01F1E2CF0EA0
:101B1000D11C08C08091F100F60181936F01015042
:101B2000110969F08091E80085FDF4CF8091E8000B
:101B30008B778093E8000E94BD19882399F391E088
:101B400001C090E08091E8008B778093E8009923B2
:101B500009F404CD89A1853009F447C048F48130E7
:101B600001F190F0823009F4F9CC843029F13FC0C2
:101B70008730C9F1D0F18830C1F18E3FC1F589833A
:101B800093E09A838B8313C019828CE0E8E4F1E040
:101B9000DE01129601900D928A95E1F78EEF8D8706
:101BA00006C08093CC0284E089838EEF8A83CE01C5
:101BB00001960E941A1AD2CC8091CC02882309F493
:101BC000CDCC8AA1811104C08BA10E949E27C6CCD6
:101BD00081E090E00BA002C0880F991F0A94E2F701
:101BE0000E947627BBCC85E003C084E001C08FEF64
:101BF0000E941A23B3CC09BD19BD09B400FEFDCF64
:101C00008091D8008F7D8093D8008091E000826021
:101C10008093E0008091E00081FDFCCF10929E0255
:101C20000E94DD27A6CC232B09F081CEB6CE213928
:101C3000314008F0C8CEFDCE80E0089590919B021F
:101C400092FF10C041E0282F2471243009F040E0B9
:101C500031E0282F2871283009F030E0431711F0C7
:101C60002CE0822793FF10C041E0282F24712431FB
:101C700009F040E031E0282F2871283109F030E0E8
:101C8000431711F02CE0822730919C0230FF10C0E6
:101C900051E0282F2171213009F050E041E0282F38
:101CA0002871283009F040E0541711F029E082270C
:101CB00031FF10C041E0282F2171213109F040E0AF
:101CC00031E0282F2871283109F030E0431711F056
:101CD00029E0822794FD877E08958238910569F175
:101CE000B0F48133910509F475C048F48932910547
:101CF00009F467C08A32910509F471C008958533EB
:101D0000910509F459C089339105B9F00895833ECE
:101D1000910589F138F4803E9105D1F0823E91051C
:101D200029F10895863E9105C9F1873E9105D9F1C3
:101D3000843E910509F06CC027C020919B0220FDD4
:101D400057C021FD55C020919C0223FD5BC0089522
:101D500080919B0280FD48C080919C0280FF48C01A
:101D600080919B0284FD46C083EE51C080919B020E
:101D700082FF3CC0F5CF80919B0282FD37C08091ED
:101D80009C0280FD35C0ECCF80919C0281FF36C063
:101D900080919B0284FD2EC087EE39C080919B020A
:101DA00083FF2AC0F5CF80919B0283FD25C08091DF
:101DB0009C0281FD23C0ECCF80919B0285FD22C057
:101DC0001FC080919B0285FD1BC080919C0283FFF8
:101DD00019C00AC080919B0286FD16C017C0809171
:101DE0009B0286FD13C010C089E311C082EE0FC0B4
:101DF00080EE0DC080E00BC086EE09C084EE07C007
:101E000085E305C089E203C08AE201C081E390E076
:101E1000089520916F029091360257E02917A9F09A
:101E200030E0529FF001539FF00D1124E95CFD4F0B
:101E30007181761306C07081781303C075817413A5
:101E400006C02F5F3F4F2770E9CF80E0089581E003
:101E500008957E30B0F46630A0F48230A0F494E5AA
:101E6000899FF001112486E0789FE00DF11D112477
:101E7000E60FF11DEE0FFF1FEF50FE4F859194917D
:101E8000089580E001C081E090E008951F93CF9312
:101E9000DF930E946D0EEC01C11580E5D807E8F5CF
:101EA000C11590E4D90708F0A8C0C03ED10530F5AF
:101EB000CD3CD10508F094C0C83AD10578F4C53AB4
:101EC000D10508F083C0C130D10509F47CC008F405
:101ED000F2C0C430D10508F0F1C0EDC0C33CD1055B
:101EE00008F0E9C0C85AD0E0CC0FDD1FC95ADE4F58
:101EF0000990D881C02DCE019464E1C0C11580E263
:101F0000D80708F0CBC0C11591E0D90708F06BC025
:101F1000C83ED10508F4D2C0CEC0C03682E5D8078D
:101F200028F5C03492E5D90708F079C0C03282E5BF
:101F3000D80708F06CC0C11592E5D90708F481C034
:101F40004C2F4695469580E2489FA0011124C3700E
:101F500021E030E0C90102C0880F991FCA95E2F75D
:101F6000EA01C82BD92BCE019D68A9C0C03A82E5F1
:101F7000D807B8F48C2F8F71C03892E5D90708F0D4
:101F80007BC08695869590E2899F90011124C3704D
:101F900081E090E002C0880F991FCA95E2F79A6825
:101FA00068C0C03C82E5D80708F46DC0C03E92E529
:101FB000D90708F080C0CF71DD27DC2FCC27CE01F8
:101FC000806F906A7CC081E090E079C0C55AD0E013
:101FD000CC5ADE4F8881C82FD0E0CE0190646FC00C
:101FE000CE0190656CC08D2F0E941E0E182FCE0161
:101FF00099270E946D0E1F715CC0CE0199270E9427
:102000006D0ECC27DF70D06A8C2B9D2B58C0CF7102
:10201000D0E0DC2FCC27CE01816F906A50C08C2F8E
:102020008F718695869590E2899F90011124C370E7
:1020300081E090E002C0880F991FCA95E2F79C6882
:1020400018C08C2F8F710E941E0E95E0D695C795F3
:102050009A95E1F7CF70D0E0DC2FCC27282F30E025
:1020600084FF05C084E0220F331F8A95E1F7D06911
:10207000CE01822B932B23C090E0D82FCC27CE010A
:10208000846F906A1CC08C2F8F710E941E0E8F71FE
:1020900090E0D82FCC27CE01906211C08D2F8F7188
:1020A0000E941E0E182FCE0199270E946D0E1F71DF
:1020B0009062912B04C080E090E001C0CE01DF91DE
:1020C000CF911F910895A8E0B0E0E9E6F0E10C940B
:1020D0003E2B66EE7EEF80E090E00E94032C60E0F5
:1020E00082E090E00E94E52B60E083E090E00E94B7
:1020F000E52B1092920260E074E184E090E00E948F
:10210000032C60E086E090E00E94E52B6FEF87E013
:1021100090E00E94E52B40E050E0BA0188E090E0BA
:102120000E94F72B60E084E290E00E94E52B60E0E3
:1021300087E190E00E94E52B60E08CE090E00E9457
:10214000E52B60E08DE090E00E94E52B19821A8279
:102150001B821C821D821E821F82188648E050E06E
:1021600068E170E0CE0101960E94D52B40E050E07E
:10217000BA0180E290E00E94F72B1092D9011092F0
:10218000DA011092DB011092DC0184E08093D90126
:102190004091D9015091DA016091DB017091DC012D
:1021A0008FE090E00E94F72B40E050E0BA0183E11D
:1021B00090E00E94F72B2896E2E00C945A2B809531
:1021C0009091680389238093680308958095909186
:1021D0009E02892380939E02089590919E02809191
:1021E0006803982B90930F02809191028823D9F075
:1021F000892B80930F0280913401882331F08091E4
:102200009B0287FF02C08EE101C086E0E1E1F2E0BF
:1022100090E0815028F021912223D9F39F5FF9CFDC
:1022200091111092910240E250E061E772E08FE07C
:1022300092E00E94242E892B21F180E2EFE0F2E06F
:10224000A1E7B2E001900D928A95E1F7E0916D036C
:10225000F0916E033097A9F080913401882359F0F2
:1022600080919B0287FF07C080910F02809310022C
:1022700086E080930F020280F381E02D8FE092E0F0
:10228000099508959091700280958923809370023A
:10229000282F277069F4981759F090919C0292FFAB
:1022A00007C08695869586950E949E27109270029B
:1022B000089590919C0292FB222720F9281779F02B
:1022C00080FB92F990939C0260919B0270919C021A
:1022D00084E090E00E94032C82E00E944211089565
:1022E00080916F0290913602891719F08F5F877085
:1022F000FBCF08950F931F93CF93DF938091350207
:1023000082958F7009F052C080913402882309F4BD
:102310004DC080916F024091360250913002109171
:102320002F026091310270913202C0913801D09138
:10233000390107E08417D1F190E0089FF001099F6F
:10234000F00D1124DF01A95CBD4F14962C91149758
:10235000222349F111962C911197251324C02C9119
:10236000211321C015962C91159721111CC012968E
:102370002D913C911397261B370B2C173D0798F492
:10238000809135028F70806180933502E35CFD4F50
:1023900080818F70806180838FE292E00E94BB0316
:1023A0000E94701103C001968770C4CFDF91CF9156
:1023B0001F910F910895A4E1B0E0E1EEF1E10C94DA
:1023C000342B8C0186E0F801DE011F9601900D92FE
:1023D0008A95E1F7D80114968C9114971596EC9094
:1023E0009FE2A92E92E0B92E90913302911121C063
:1023F000882309F463C1EE2009F447C0C8010E9494
:10240000BA27F82E882309F440C087E0F801D501E7
:1024100001900D928A95E1F780913302813031F479
:1024200080912F02909130020E9400270E947A1121
:1024300054C1F80190808180C280D380F090340232
:10244000409131025091320220913801309139018E
:10245000FF2009F4E0C0B601641B750B6217730717
:1024600008F099C0882309F438C180913502282FDB
:10247000207F90913002222361F0981509F45CC00E
:10248000C8010E94BA2781115FC0C8010E94BB0326
:1024900015C1981114C090912F02991110C0E1102C
:1024A0000EC08F708061809335028FE292E00E94AF
:1024B000BB0380913502D80116968C930DC1E110B3
:1024C00035C040E0682D892D0E94090FE82E81114A
:1024D000F8C09F86888A8F8598890E940027292FB7
:1024E00022952F70243020F49F70223028F009C0EC
:1024F0002A50223080F014C0992349F0811107C07E
:1025000013C0992321F0F8019681907F69F0805ED5
:10251000883030F409C0803F38F0815F833020F08C
:10252000C8010E94BB03EF2CFE2CD7C0809135025E
:10253000816080933502C5C090912F029911A0CF80
:10254000E1109ECFF80199C0EE2009F49ECF2091B2
:102550003502822F82958F7090E002978CF08091E7
:102560002F029091300299878887DB86CA868091F6
:1025700033028C871D862E87CE0108960E94BB03EE
:1025800087E0F801AFE2B2E001900D928A95E1F7A1
:102590000E947A1193C090913502292F207F39F43F
:1025A0008FE292E00E94BB0387E0D50192C08823AE
:1025B00009F493C08091300288110CC080912F02E1
:1025C000891108C0E11006C0F8019683C8010E9475
:1025D000BB036EC0C8010E94BA27882309F455CFF7
:1025E000EE2009F452CF20913502822F82958F7010
:1025F00090E002972CF280912F02909130029A8302
:102600008983DC82CB82809133028D831E822F836B
:10261000CE010196B3CFC41AD50AC216D30608F06C
:1026200047C0882309F44AC0FE2CEE2009F42DCFC0
:102630008091300288112EC080912F0289112AC00A
:10264000B8ECCB16D104E8F48091350280FD19C0B6
:1026500082958F70482F50E04115510591F02091DF
:102660003502F80126834F30510541F08F5F982FD6
:102670009295907F822F8F70892B8683C8010E944C
:10268000BB0387E0F801AFE2B2E001900D928A95BA
:10269000E1F723C0C8010E94BA27811171CF809150
:1026A0003502816080933502C8010E94BB0315C0CA
:1026B00087E0D5011D928A95E9F70FC0FF24F394B6
:1026C0000CC08FE292E00E94BB03EFE2F2E087E0F1
:1026D000DF011D928A95E9F7F12C8F2D6496ECE0CD
:1026E0000C94502BA0E0B0E0E8E7F3E10C94382B19
:1026F00080913B0190913C01892BB9F0809195022A
:102700008F5F80939502811110C00E940B1D90E095
:1027100090933C0180933B01892B39F40E94821DE8
:1027200081E080933A010E9445230DED11E078018C
:10273000D0E0C0E087E0C82ECC0E8C2F0E94F21DA6
:102740008C2D0E94F21D8C2F0E94551E8F73F70155
:102750009081891721F08083DD24D39401C0D12C8E
:102760008C2D0E94551E8F73F7019781891719F0E0
:10277000878381E001C080E0D82ADD290E94461EBF
:10278000CF5FFFEFEF1AFF0AC730A1F610929A024F
:10279000C0919902CC2309F47DC00E947B21209135
:1027A000970230919802AC01421B530B9A0190930F
:1027B0009802809397024F3F510509F018F4452B7A
:1027C00019F102C02FEF30E0109299021092960298
:1027D000E091D701F091D801AF01425F5F4F90E0E7
:1027E00030E08081882341F0281718F010829C2F58
:1027F00003C0821B80833C2F3196E417F50789F7CD
:102800003093990290939602DD23B1F110929602D3
:10281000E091D701F091D80180919A0290919902AC
:10282000AFEEB1E0AF01425F5F4F6EE1E80128819A
:102830003C91321779F0308131110CC060832C93B8
:1028400098819227282F30E0292B81E0232B09F44F
:1028500080E091E0319611960F5F1F4FE417F50766
:1028600029F780939A029093990280919A02CDB7AA
:10287000DEB7E8E00C94542B81E090919602992306
:10288000A1F38111C3CF0E947B2190939802809382
:102890009702BCCFD111F7CF80E0EFCFA6E0B0E038
:1028A000E4E5F4E10C943C2B0E947B218C018091A7
:1028B0009302909194020817190781F019821A82E5
:1028C0000E947B21682F49815A81792F80E090E016
:1028D0000E94B61B10939402009393022696E4E0A4
:1028E0000C94582B8091C40287FF11C08091E8009E
:1028F00082FD05C08091CE028111F8CF11C0809178
:10290000E8008B770BC08091CE02882349F080913C
:10291000E80080FFF8CF8091E8008E778093E80090
:102920000895982F973068F59093E900981739F03B
:102930007091EC002091ED005091F00003C0242F25
:10294000762F50E021FD02C09F5FECCF3091EB006D
:102950003E7F3093EB003091ED003D7F3093ED00F2
:102960003091EB0031603093EB007093EC002093DA
:10297000ED005093F0002091EE0027FDE5CF80E0C0
:1029800008958F708093E90081E008952091CA0234
:102990003091CB022617370748F06115710539F4DD
:1029A0002091E8002E772093E80001C0B901FC01D6
:1029B00020E06115710579F18091CE028823F1F153
:1029C0008530F1F18091E80083FD3CC08091E80002
:1029D00082FD2EC08091E80080FFEBCF2091F300B4
:1029E0008091F20090E0922B6115710551F08830D2
:1029F000910538F421912093F100615071090196FD
:102A0000F3CF21E0089709F020E08091E8008E776D
:102A10008093E800CECF2111CFCF0AC08091CE02A3
:102A2000882361F0853061F08091E80083FD0AC061
:102A30008091E80082FFF2CF80E0089582E008955F
:102A400083E0089581E0089543E050E0BC0185E013
:102A50000E942221089545E050E0BC0182E00E94DE
:102A600022210895CF93DF93EC01809134018111ED
:102A700005C048E050E0BE0181E00BC080919B02A0
:102A800087FF03C040E285E002C048E081E050E0FB
:102A9000BE010E94222180E2FE01A1EAB2E0019083
:102AA0000D928A95E1F7DF91CF910895AAE2B0E007
:102AB000ECE5F5E10C943D2BE4ECF2E08CEC92E0DB
:102AC0002091F10021938E179F07D1F78091C502C5
:102AD000833009F463C030F4813071F0823009F43E
:102AE0009FC0B6C08A3009F48BC08B3009F46EC029
:102AF000893009F0ADC020C08091C402813A09F04C
:102B0000A7C08091E800877F8093E8008091C80289
:102B10009091C902892B21F460E281EA92E003C01E
:102B200060E080E090E070E00E94C6148091E800D0
:102B30008B778093E8008CC08091C402813209F0C9
:102B400087C08091C8029091C902009719F003973D
:102B500009F07EC08091E800877F8093E800809133
:102B6000E80082FD05C08091CE028111F8CF70C0CF
:102B70002091F3008091F20090E0922B029731F4C3
:102B80008091F100813011F0863021F48091F100C4
:102B90008093A0028091E8008B7756C08091C40298
:102BA000813A09F055C08091C8029091C902892BE1
:102BB00009F04EC08091E800877F8093E800809103
:102BC000E80080FFFCCF8091340139C08091C402BD
:102BD0008132F1F58091C8029091C902892BC1F52B
:102BE0008091E800877F8093E8000E9472148091B2
:102BF000C6028093340110929E020E94DD2728C0F5
:102C00008091C402813221F58091E800877F809312
:102C1000E8000E9472148091C70280939F0218C03E
:102C20008091C402813AA1F48091E800877F80936B
:102C3000E8008091E80080FFFCCF80919F028093A4
:102C4000F1008091E8008E778093E8000E94721472
:102C50008091E80083FFE4C18091C4029091C50295
:102C6000492F50E04A30510508F0DAC1FA01E25824
:102C7000FF4F0C94AA2C803821F0823809F0D0C183
:102C800008C08091C1029091C202992389F08260AC
:102C90000FC08091C8028F70873008F0C1C1809347
:102CA000E9008091EB0085FB882780F91092E9000C
:102CB0009091E800977F9093E8008093F100109244
:102CC000F10070C1282F2D7F09F0AAC1882319F0C7
:102CD000823061F0A5C18091C602813009F0A0C1A7
:102CE000933009F080E08093C2022EC08091C6022A
:102CF00081112AC08091C8028F702FEF280F2630D3
:102D000008F08EC18093E9002091EB0020FF1CC0E9
:102D1000933021F48091EB00806214C09091EB001D
:102D200090619093EB0021E030E0A90102C0440FD4
:102D3000551F8A95E2F74093EA001092EA008091CD
:102D4000EB0088608093EB001092E9008091E8002E
:102D5000877F8093E8000E94721462C1811160C174
:102D60001091C6021F778091E3008078812B8093B9
:102D7000E3008091E800877F8093E8000E9472144E
:102D80008091E80080FFFCCF8091E3008068809311
:102D9000E300111102C082E001C083E08093CE0203
:102DA0003FC18058823008F03BC12091C60230916B
:102DB000C7022C3D53E0350779F583E08A838AE228
:102DC00089834FB7F894DE01139620E03EE051E28C
:102DD000E32FF0E050935700E49120FF03C0E29509
:102DE000EF703F5FEF708E2F90E0EA3010F0C796E3
:102DF00001C0C0968D939D932F5F243149F74FBF3B
:102E00008091E800877F8093E8006AE270E0CE015D
:102E100001960E94C614B4C08091C8029091C90264
:102E2000432F552743305105A9F068F4413051052F
:102E300009F405C14230510509F0F2C084E790E081
:102E4000EBE5F4E04BC04132510529F14232510526
:102E500089F1E6C0C901992781309105A1F058F0A8
:102E6000029709F0DDC0E1EEF4E0E4918E2F90E0EE
:102E7000E1EEF4E030C0EFE2F5E0E4918E2F90E077
:102E8000EFE2F5E028C0E5E0F5E0E4918E2F90E078
:102E9000E5E0F5E020C08430910508F0C1C0880F5E
:102EA000991FFC01E756FE4F0190F081E02D89E06B
:102EB00090E014C08430910508F0B2C0FC01EE0F20
:102EC000FF1FEF56FE4F0190F081E02DDC01A3576C
:102ED000BE4F8C9190E0009709F4A2C02091E800C9
:102EE000277F2093E8002091CA023091CB02281757
:102EF000390708F4C90140E0009789F12091CE021A
:102F0000222309F43DC02530D9F12091E80023FDAA
:102F100037C02091E80022FD2FC02091E80020FF5B
:102F2000EBCF4091F3002091F20030E0342B00977A
:102F300059F02830310540F444914093F100319626
:102F400001972F5F3F4FF3CF41E02830310509F063
:102F500040E02091E8002E772093E800CDCF41118A
:102F6000CDCF0AC08091CE02882351F0853041F048
:102F70008091E80083FD04C08091E80082FFF2CFD9
:102F80008091E8008B778093E8004AC0803809F090
:102F900047C08091E800877F8093E8008091C3025A
:102FA0008093F1008091E8008E77D3CE811138C0F4
:102FB0008091C6029091C702992702978CF5809163
:102FC000E800877F8093E8001091C6021093C30247
:102FD0000E947214111106C08091E30087FD02C0A7
:102FE00081E001C084E08093CE0242E061EC81E0A8
:102FF0000E94911442E061EC82E00E94911442E24E
:1030000061EC85E00E94911442E261EC83E00E9451
:10301000911442E260EC84E00E9491148091CE020F
:103020008091E80083FF10C08091E800877F809343
:10303000E8008091EB0080628093EB0005C082E1A4
:1030400090E0EFECF4E04ACFAA96E3E00C94592B21
:103050001F920F920FB60F9211242F933F934F930D
:103060005F936F937F938F939F93AF93BF93CF9310
:10307000DF93EF93FF93C091E900CF708091EC0054
:10308000D82FD17080FDD0E81092E9008091F00037
:10309000877F8093F00078940E9456151092E90083
:1030A0008091F00088608093F000CD2BCF70C093AA
:1030B000E900FF91EF91DF91CF91BF91AF919F9187
:1030C0008F917F916F915F914F913F912F910F90D1
:1030D0000FBE0F901F901895E8EDF0E080818E7F75
:1030E00080831092E2001092DA001092E100A0EECC
:1030F000B0E08C9181608C9380818F77808319BC44
:10310000A7EDB0E08C918E7F8C9380818F7E808341
:1031100010929D020895A0E0B0E0E1E9F8E10C947E
:10312000382BC8EDD0E088818F7E8883E7EDF0E012
:1031300080818160808384E082BF81E080939D02F2
:1031400088818E7F888302EE10E0F8011082109251
:10315000DA0081EEC82ED12CF601108288818F779B
:10316000888388818068888388818F7D888319BC63
:103170001092CE021092C3021092C2021092C102AB
:1031800090EEE92EF12CF70180818B7F808388817E
:103190008160888342E060E080E00E949114F60143
:1031A00080818E7F8083F80180818160808380812F
:1031B00088608083F70180818E7F80838881806131
:1031C0008883CDB7DEB7E8E00C94542B1F920F92A2
:1031D0000FB60F9211242F933F934F935F936F93EA
:1031E0007F938F939F93AF93BF93EF93FF938091C0
:1031F000E10082FF09C08091E20082FF05C080915A
:10320000E1008B7F8093E1008091DA0080FF2AC08B
:103210008091D80080FF26C08091DA008E7F809355
:10322000DA008091D90080FF18C080E189BD82E179
:1032300089BD09B400FEFDCF81E08093CE0280916C
:103240009D0281110FC00E946C180E948B18809102
:10325000E20084608093E20005C019BC1092CE02A7
:1032600010929D028091E10080FF17C08091E200E2
:1032700080FF13C08091E2008E7F8093E2008091F6
:10328000E20080618093E2008091D80080628093A8
:10329000D80019BC85E08093CE028091E10084FFC4
:1032A00030C08091E20084FF2CC080E189BD82E1C2
:1032B00089BD09B400FEFDCF8091D8008F7D809339
:1032C000D8008091E1008F7E8093E1008091E20040
:1032D0008F7E8093E2008091E20081608093E20023
:1032E0008091C302882311F084E007C08091E3003D
:1032F00087FD02C081E001C083E08093CE0280910F
:10330000CE028091E10083FF27C08091E20083FF1D
:1033100023C08091E100877F8093E10082E0809369
:10332000CE021092C3028091E1008E7F8093E10073
:103330008091E2008E7F8093E2008091E2008061C4
:103340008093E20042E060E080E00E94911480916E
:10335000F00088608093F000FF91EF91BF91AF91F2
:103360009F918F917F916F915F914F913F912F919D
:103370000F900FBE0F901F9018952091E400309190
:10338000E50095E64091EC00842F817040FF23C05A
:103390008091E80080FD1DC08091CE02882399F0C5
:1033A000853099F08091EB0085FD11C04091E400DB
:1033B0005091E5002417350729F3915011F09A0137
:1033C000E1CF84E0089582E0089583E0089581E0EC
:1033D000089580E008954091E80042FFDDCF089510
:1033E000EF92FF920F931F93CF93DF937C018B019A
:1033F0000E94BD19811119C0E70101151105A1F045
:103400008091E80085FD0AC08091E8008E77809366
:10341000E8000E94BD19882381F307C08991809339
:10342000F10001501109E9CF80E0CDB7DEB7E6E049
:103430000C94562BCF932091CE02243011F5C091DD
:10344000E900CF703091EC00232F217030FD20E88F
:10345000C22B23E02093E9002091E80020FF0EC05A
:1034600040E050E060E270E00E94F019811110929B
:10347000CC028091E8008E778093E800CF70C093F3
:10348000E900CF9108959C013A9521153F4130F50F
:10349000BC0166277270AC01442754709C0122273E
:1034A000387094FF0FC090FF02C080E101C080E03F
:1034B000672B09F08062452B09F08064232B79F09B
:1034C00080680895892F8170672B09F08260452BF1
:1034D00009F08460232B19F08860089580E0089536
:1034E000FC018281813039F4958192FD12C090FFF8
:1034F00010C082E00895823039F4858182FD06C0D3
:1035000080FD06C083E0089586E0089585E0089573
:1035100084E00895CF93DF93EC010E940429CE014B
:10352000805E9109089710F0209731F4CE010E9437
:10353000431A0E941B2805C0CE010E94431A0E9414
:103540000A28DF91CF9108958FE39CE90197F1F765
:1035500000C000008091D202833029F0853031F024
:10356000813041F403C081E990E002C080E990E03D
:103570000E948A1A1092D20208958FE39CE9019763
:10358000F1F700C000008091D002833029F085302F
:1035900031F0813041F403C08BEA90E002C08EEA42
:1035A00090E00E948A1A1092D0020895CF93DF9380
:1035B000EC01805E9109089710F0209731F4CE015C
:1035C0000E94431A0E94222805C0CE010E94431A7D
:1035D0000E9411288C2F0E946829DF91CF910895B5
:1035E0000F931F93CF93DF938C01C99719F0C0E01D
:1035F000D0E002C0C0E5D0E0C8010E94D61A2097F2
:1036000041F08FE99FE00197F1F700C0000021979A
:10361000F6CFC8010E948A1ADF91CF911F910F91B6
:103620000895CF93DF93EC018A81833061F480E9C0
:1036300090E00E94F01A80E990E00E94F01A80E980
:1036400090E00E94F01A8A81843020F080E990E0B6
:103650000E94F01ADF91CF910895CF93DF93EC0190
:103660008A81833061F48EEA90E00E94F01A8EEA3B
:1036700090E00E94F01A8EEA90E00E94F01A8A818F
:10368000843020F08EEA90E00E94F01ADF91CF9112
:1036900008950E94701A8093D202833029F08530F9
:1036A00031F0813061F407C081E990E006C080E923
:1036B00090E00E94F01A80E990E00E94D61A0895E6
:1036C0000E94701A8093D002833029F0853031F047
:1036D000813061F407C08BEA90E006C08EEA90E08A
:1036E0000E94F01A8EEA90E00E94D61A0895982F50
:1036F00092959F7019F0892F24E001C020E0982F47
:103700009695969511F02E5F892F982F969509F032
:103710002F5F822F0895A6E0B0E0E1E9FBE10C9471
:103720003D2B26E0FC01DE01119601900D922A95B9
:10373000E1F7FC01258189819A81222359F06623D2
:1037400049F00E94D126182F682F89819A810E9402
:10375000412703C00E940D27182F69817A81812F8C
:103760000E94290F2696E3E00C94592BA4E3B0E0C5
:10377000ECEBFBE10C943D2B4FA758AB69AB7AAB5C
:103780008BAB9CAB911110926803CE01889627E019
:10379000DC011D922A95E9F726E0FE01BF96DC01C7
:1037A00001900D922A95E1F72CA52223C1F061E04A
:1037B0000E948B1B8091CC02882389F08DA58111FA
:1037C00002C087E001C086E0898388A58A8389A535
:1037D0008B838EEF8C83CE0101960E941A1A87E0AC
:1037E000FE01B896DE01919601900D928A95E1F75F
:1037F000CE0181960E94DB1181112CC087E0FE0171
:10380000B196DE01119601900D928A95E1F76DA1B6
:10381000662301F12091360230E0C90101968770DC
:10382000992740916F0250E08417950761F16D83ED
:1038300097E0929FD001939FB00D1124A95CBD4FDA
:10384000FE01319601900D929A95E1F78093360230
:103850000E94701117E080916F02909136028917D3
:1038600009F1189FC0011124895C9D4F0E94DB1152
:103870008823C1F080916F0290E0019687709927AC
:1038800080936F02E8CF10929E020E94DD27109273
:10389000360210926F02EFE2F2E087E0DF011D9244
:1038A0008A95E9F7E496E3E00C94592B10929E0276
:1038B0000E94DD272FEF84E39CE021508040904060
:1038C000E1F700C000009AE088E10FB6F894A895EF
:1038D000809360000FBE90936000FFCF8F929F9205
:1038E000AF92BF92CF92DF92EF92FF920F93CF935E
:1038F000C82F0E94771B56985E9825982D98269879
:103900002E9827982F98482F50E0FA013197E730EA
:10391000F105B0F4E857FF4F0C94AA2C259A2D9A84
:1039200011C0259A2D9A269A2E9A22C0259A2D9A50
:1039300004C0259A2D9A269A2E9A279A2F9A18C053
:103940008130B1F48091CE01811159C080915D0325
:10395000816080935D0360E086950E944E2660E062
:1039600081E00E944E2620E04FEF6FEF8CEB42C0CB
:103970008091CE01811143C088E090E00E94C92B64
:103980004B015C0184E290E00E94C12B282F30E0C3
:1039900040E050E060E070E080E090E000E20E94F3
:1039A000BF2C282939294A295B2920935D033093AC
:1039B0005E0340935F0350936003609361037093D1
:1039C0006203809363039093640320FF16C0822FE9
:1039D000816080935D0386950E94912680915D03AE
:1039E00086950E94912621E04091600360915F03DB
:1039F00080915E030E94212502C00E9456248C2FD4
:103A0000CF910F91FF90EF90DF90CF90BF90AF904C
:103A10009F908F90089580E290E090933C01809376
:103A20003B018091820381110EC00E944A2A81E0ED
:103A3000809382032FEF83ED90E3215080409040EC
:103A4000E1F700C0000060E570E080E40E94502AC9
:103A500090933C0180933B01892B09F04EC060E5B7
:103A600070E080E00E94C32A90933C0180933B0168
:103A7000892B09F042C060E570E080E00E94C32A13
:103A800090933C0180933B01892BB9F560E570E090
:103A90008FE30E94C32A90933C0180933B01892BC2
:103AA00061F50E94162B60E570E080E40E94502AC8
:103AB00090933C0180933B01892BF9F460E570E021
:103AC0008CE00E94C32A90933C0180933B01892B98
:103AD000A1F460E570E080E00E94C32A90933C016D
:103AE00080933B01892B49F460E570E08FE30E94ED
:103AF000C32A90933C0180933B010E94162B809136
:103B00003B010895CF93DF9356985E9825982D98A2
:103B100026982E9827982F98C8E8D0E08FEF90E04D
:103B200099838883AAE8B0E011969C938E93ECE881
:103B3000F0E091838083259A2D9A2FEF80E792E021
:103B4000215080409040E1F700C00000269A2E9A54
:103B50002FEF80E792E0215080409040E1F700C0D5
:103B60000000279A2F9A2FEF80E792E021508040A3
:103B70009040E1F700C0000025982D982FEF80E7D6
:103B800092E0215080409040E1F700C0000026986C
:103B90002E982FEF80E792E0215080409040E1F78F
:103BA00000C0000027982F988091D90187702FEFCF
:103BB000829FC001112495958795959587959927A2
:103BC0009983888311969C938E93918380835698D2
:103BD0005E9825982D9826982E9827982F98DF91F3
:103BE000CF910895CF93E82F873080F580913B01E6
:103BF00090913C01892B09F047C0CE2F60E570E021
:103C000080E40E94502A90933C0180933B01892BD1
:103C1000D1F460E570E082E10E94C32A90933C01F8
:103C200080933B01892B79F481E090E001C0880FFB
:103C3000CA95EAF760E570E080950E94C32A9093E8
:103C40003C0180933B010E94162B1EC090E0FC01BA
:103C50003797E730F105C0F4E157FF4F0C94AA2CD9
:103C6000209A289811C0219A29980EC0229A2A9841
:103C70000BC0239A2B9808C0529A5A9805C0539AA1
:103C80005B9802C03E9A4698CF9108952098289854
:103C90002198299822982A9823982B9852985A98D4
:103CA00053985B983E9846980895CF93873040F597
:103CB00080913B0190913C01892B59F560E570E0C2
:103CC00081E40E94502A90933C0180933B01892B10
:103CD00011F0C0E011C080E590E00E94F22A97FF49
:103CE00005C090933C0180933B01F3CFC82FC09552
:103CF00010923C0110923B010E94162B8C2F0AC09F
:103D00009FB18FB1807F869586959370892B809522
:103D100001C080E0CF9108958098889A8198899A0F
:103D200084988C9A85988D9A86988E9A87988F9A7F
:103D300008958091A00208950895A0E0B0E0E3EA1C
:103D4000FEE10C94332BFC018280748081E084833B
:103D5000E3E3F5E09490E2EBF5E0E4910091600399
:103D60000695015810E0000F111F012F1127C2E125
:103D7000D3E026EDC22E22E0D22EAA24AA94B12CA2
:103D8000E919EE2EF12C22E0281530F080915E0327
:103D9000888380915F038983711003C01B821A821C
:103DA0004AC08B818823F9F081508B832FEF829F4B
:103DB000C00111246C8170E00E941A2BFB01FF27C7
:103DC000ED5CFA4F8491E82FE9192FEFE29FC001D3
:103DD0001124B7010E941A2B80916003689FB001E3
:103DE00011247A8328C00E94B12BB5010E94962C21
:103DF0008017910704F582E0881588F40E94B12BA2
:103E0000B5010E94962C88830E94B12B20915F03FC
:103E10002695622F70E00E94962C280F29831A8223
:103E200080916003843120F0893C18F088EC01C057
:103E300084E18C838B8396014A81698188810E9409
:103E40007C24259624E0C20ED11C83E0CD35D80712
:103E500009F099CF0E944523CDB7DEB7EDE00C9471
:103E60004F2BEF92FF920F931F93CF93DF938C0111
:103E7000C6EDD2E0E12CF12CF8018481F7E0EF16D9
:103E8000F1041CF4882339F002C0811104C09E01A2
:103E90004091600302C09E0140E060915F03809109
:103EA0005E030E947C248FEFE81AF80A24969FE0B4
:103EB000E916F10409F70E944523F801848190E096
:103EC0000196817099278483CDB7DEB7E6E00C9424
:103ED000562BA0E0B0E0EFE6FFE10C94342BEC01B0
:103EE0004C81042F10E09801D8010E946D2C9B0199
:103EF000AC010E94382C6B017C01E0E2F0E0E01B99
:103F0000F10BA5E5B0E09B01AC010E94382C4B0100
:103F10005C019F01DF010E94B02C9B01AC010E945B
:103F2000432C9B01AC012C0D3D1D4E1D5F1DC50199
:103F3000B4010E944B2C822FF22E99E2921728F0A6
:103F400093E0299F900111240DC025E530E0281B46
:103F50003109C901880F991F280F391F37FF02C087
:103F60002F5F3F4F35952795122F109596EDC92E4F
:103F700092E0D92E00E085E5E82EEF1801FD02C0A1
:103F80008E2D01C08F2D9601412F60915F030E94FD
:103F90007C240F5F84E0C80ED11C0F3079F70E949B
:103FA00045238C81811102C091E003C0803219F455
:103FB0009FEF9093370190913701890F8C83CDB794
:103FC000DEB7ECE00C94502B0F931F93CF93DF934D
:103FD000C6EDD2E0FE011182108212821382349665
:103FE00083E0E231F807B9F700E010E08091D402F5
:103FF000082E000C990B0817190794F080913601D0
:10400000082E000C990B8017910754F09E014091E7
:10401000600360915F0380915E030E947C2404C072
:10402000198218821A821B820F5F1F4F24960F304D
:104030001105E1F60E944523809135019091D4024B
:10404000980F9093D40220913601280F20933601C7
:10405000121614F49E301CF0819580933501DF9187
:10406000CF911F910F910895A0E0B0E0EAE3F0E254
:104070000C94372BFC01828180FF03C0DD24DA948D
:1040800002C0DD24D39406ED12E0C0E0D0E02FE0C2
:10409000B22EF801118210821282138294E0E92E6E
:1040A000F12CC12C8091D3028C0D80312CF06B2D22
:1040B0000E94882C892F02C087FD815F082E000C8A
:1040C000990BC817D90791F4809160038E9DA001C8
:1040D0008F9D500D112455954795559547959801FD
:1040E00060915F0380915E030E947C24CD0CF1E01F
:1040F000EF1AF108B9F621960C5F1F4FCF30D105AA
:1041000041F60E9445238091D30291E0D91206C066
:10411000811102C08EE007C0815005C090E0019679
:10412000BE010E94962C8093D302CDB7DEB7E9E0A2
:104130000C94532BEF92FF921F93CF93DF93EC01DC
:1041400086EDE82E82E0F82E10E08C8197014091F8
:10415000600360915F03810F0E947C241F5E84E0F6
:10416000E80EF11C1F3F89F70E9445239A818C813C
:1041700090FF02C08F5F01C081508C83DF91CF918F
:104180001F91FF90EF900895A4E0B0E0EAECF0E218
:104190000C943C2B8C018091D50281110AC09E01A8
:1041A0002F5F3F4F4FEF6FEF0E947C248A818093F7
:1041B000D502F8018481813051F028F0823061F419
:1041C0004091D5020AC08091D50240E007C06091BD
:1041D000D50240E080E003C040E080E060E00E9463
:1041E000D723F801848190E0019663E070E00E949B
:1041F000962C84832496E4E00C94582BCF93DF9381
:10420000EC01EDE5F3E0438162818C810E94092598
:104210008C818F5F8C83DF91CF910895CF93DF9353
:10422000EC01EC81F0E0ED5CFA4F4491EDE5F3E058
:10423000628181810E9409258C818F5F8C83DF914F
:10424000CF9108959B019091CE029430F1F48F703C
:104250008093E9008FEF9091E800815095FD06C0B2
:1042600095ED9A95F1F700008111F5CF8091E80066
:1042700085FF0BC0BA01C90140E050E00E94F0196F
:104280008091E8008E778093E800089578941F92DB
:104290000F920FB60F9211248F939F93AF93BF93FA
:1042A0008091720390917303A0917403B091750390
:1042B0000196A11DB11D8093720390937303A09387
:1042C0007403B0937503BF91AF919F918F910F903D
:1042D0000FBE0F901F9018959C014FB7F8948091D6
:1042E000720390917303A0917403B09175034FBF53
:1042F000821B930B08952FB7F894809172039091CD
:104300007303A0917403B09175032FBF08951F929A
:104310000F920FB60F9211248F939F93AF93BF9379
:1043200080917103811113C0809172039091730386
:10433000A0917403B09175034196A11DB11D8093A6
:10434000720390937303A0937403B0937503BF91AA
:10435000AF919F918F910F900FBE0F901F90189566
:10436000209134012223C9F020919B0227FF15C020
:10437000262F2695269526952E31C8F4FC01E20FAE
:10438000F11D677081E090E001C0880F6A95EAF73F
:1043900080959281892382830895FC01069622816B
:1043A000621301C012823196E817F907C1F7089528
:1043B000209134012223C1F020919B0227FF14C0D9
:1043C000262F2695269526952E3130F5FC01E20FF5
:1043D000F11D677081E090E001C0880F6A95EAF7EF
:1043E0009281892B82830895FC0132962FEF30E071
:1043F0004191641789F02F3F19F4411101C0232F17
:104400003F5F3630A9F72F3F39F0FC01E20FF11D75
:1044100027FDFA95628308950895A3E0B0E0E3E1F3
:10442000F2E20C943E2B20916F0330917003281719
:104430003907A1F09093700380936F03E0916D03AF
:10444000F0916E03309751F024E029839B838A8397
:104450000680F781E02DCE01019609952396E2E0D2
:104460000C945A2BA3E0B0E0E8E3F2E20C943E2B6C
:1044700020916B0330916C0328173907A1F09093BA
:104480006C0380936B03E0916D03F0916E033097A2
:1044900051F023E029839B838A830680F781E02DF6
:1044A000CE01019609952396E2E00C945A2BE091F7
:1044B0006D03F0916E03309729F00190F081E02DAB
:1044C0000995089580E008954115510511F0FA010C
:1044D00009950895CF93DF93EC014A855B856E853E
:1044E0007F850E9464228B810E94DF108C810E9454
:1044F000E6100E94ED1086E0FE0111928A95E9F720
:10450000DF91CF910895CF93DF93EC018D8181FDF1
:1045100017C082608D83909168038B81892B809373
:10452000680390919E028C81892B80939E020E9449
:10453000ED10488559856E857F85CE010E946422E5
:1045400010926A03109269038D8180FD03C0CE0131
:104550000E946A22DF91CF9108950F931F93CF930A
:10456000DF93C42FD22FFC0185818823B1F04093C3
:1045700067030E947B21909366038093650380E22A
:104580008C0F883008F051C0C77081E001C0880FDF
:10459000CA95EAF70E94222848C080916703481311
:1045A00034C080916503909166030E946C21209134
:1045B0003801309139018217930738F510E21D0F49
:1045C000CD17B9F080E28C0F883040F4C77081E0DD
:1045D00001C0880FCA95EAF70E941B28183010F511
:1045E00081E09D2F977001C0880F9A95EAF70E948D
:1045F0002228802F0E942B2A1830B8F4D77081E02F
:1046000001C0880FDA95EAF70AC080E28C0F883083
:1046100060F4C77081E001C0880FCA95EAF70E9474
:104620001B2803C0802F0E942B2ADF91CF911F915E
:104630000F910895A0E2B0E0E0E2F3E20C943E2B8B
:104640009FEF99838A83CE0101960E941A1AA09641
:10465000E2E00C945A2B90915D0390FF04C0969574
:10466000981748F003C0811106C090E0961718F41F
:104670000E949F2608950E9491260895882311F094
:10468000FA0101C0FB0109950895EF92FF920F9383
:104690001F93CF93DF9380915D0380FF08C006EDE9
:1046A00012E082E1E82E83E0F82EF8011BC0E6ED6F
:1046B000F2E082E193E0118210821282138234963A
:1046C0008E179F07C1F7EBCF381708F4832F83832A
:1046D000381B3183281B2083981B92833496EE1657
:1046E000FF0641F0928120813181892F291760F7DF
:1046F000822FEACF80918203882381F180913B0150
:1047000090913C01892B51F580913A01882331F138
:1047100065E070E084E80E94502A892B19F010921D
:104720003A011AC0C6EDD2E065E070E088810E94CF
:10473000C32A65E070E089810E94C32A65E070E0C9
:104740008A810E94C32A65E070E08B810E94C32A9F
:104750002496EC16FD0641F70E94162B579A8BB152
:104760008F779BB190682FB7F894E016F10699F017
:10477000F80131918F0148E09BB9000000C037FF7C
:104780008BB9330F000000C000C000C08BB900C05F
:104790004A9591F7EACF2FBF8FE594E00197F1F7A3
:1047A00000C00000CDB7DEB7E6E00C94562B909128
:1047B0005D0390FF0DC0E6EDF2E0818360834283EC
:1047C0001382349693E0E231F907B9F70E9445234A
:1047D000089580915D03282F269530E0211531053D
:1047E00019F48170826005C02B32310524F081708C
:1047F000846580935D030895A0E0B0E0E2E0F4E218
:104800000C94342B49015A016B017C010E94E9236D
:104810008401A4016A2D7B2D88E090E00E94F72B93
:1048200094014A2D5B2DB601C70100E20E94DA2CEB
:10483000622F84E290E00E94E52BCDB7DEB7ECE07A
:104840000C94502B80916103882319F08150809340
:10485000610320915D0330915E0340915F035091AD
:104860006003609161037091620380916303909192
:1048700064030E94FC23089580916103833018F43F
:104880008F5F8093610320915D0330915E034091BF
:104890005F035091600360916103709162038091A6
:1048A0006303909164030E94FC230895EDE5F3E017
:1048B00020812E7F208331814281538164817581E3
:1048C000868197810E94FC2310928A030E944523CF
:1048D0000895EDE5F3E023E0208311828FEF8283DA
:1048E00083831482758130E04FEF5FEF60E0868153
:1048F00097810E94FC230895A0E0B0E0E2E8F4E292
:104900000C94362BE82EF62EE901E42FF0E061112D
:1049100006C0ED5CF94FE4914E2F2E2F71C0062F8B
:1049200010E0ED5CF94F4491F42FC42ED12C26E019
:10493000829FC00111242FEF30E0B9010E941A2B91
:104940005BEA5603C001579F900D11248E0D911DF7
:104950008E0D911D582F550F580FD901A01BB10B6B
:10496000AC9DC001AD9D900DBC9D900D1124E92F13
:10497000F59ED0011124AB2FBB277901EA1AFB0A5F
:10498000EC9CD001ED9CB00DFC9CB00D11245901A4
:10499000A51AB108A09E7001A19EF00CB09EF00C6B
:1049A0001124EF2CFF242E193F092C9D80012D9DF1
:1049B000100D3C9D100D1124212F6230710591F0D6
:1049C00048F461157105E1F061307105B9F4242FE7
:1049D0004B2F16C06430710569F040F066307105E8
:1049E00079F00CC0242F492FE12F0AC0492FEF2F57
:1049F0002B2F06C0292FE42F412F02C0292FEB2F88
:104A000049832883EA831B82CDB7DEB7EAE00C94A2
:104A1000522BA4E0B0E0EFE0F5E20C943E2B909135
:104A20005D0390FF0AC09E012F5F3F4F0E947C24D0
:104A30004B8169818A810E94D7232496E2E00C94FD
:104A40005A2BA4E0B0E0E7E2F5E20C94312BF82E0B
:104A5000762EE42E622E90915D0390FF6CC0E92FBC
:104A6000E695AE2FB0E0AF55BE4F8C918093890391
:104A70009E7F923061F49E012F5F3F4F8F2D0E94E9
:104A80007C244B8169818A810E94D7233DC082307A
:104A900019F4E090600338C0863019F4F0905E039A
:104AA00033C08930D9F3893179F5E9518E2F81707E
:104AB000582EE695F0E0ED5CF84FE4910E2F10E0F3
:104AC00086EDC82E82E0D82EA12CB12C9FE0892E35
:104AD000912CC501B4010E941A2B8F2D511002C0D8
:104AE000860F01C0861B96014E2D672D0E947C24E7
:104AF000A00EB11E84E0C80ED11C82E1C81683E06E
:104B0000D80639F70E944523F0925E0370925F0346
:104B1000E0926003662079F020915D03609161036B
:104B2000709162033F2D472D5E2D8091630390911C
:104B300064030E94FC232496EFE00C944D2BEDE5DA
:104B4000F3E043812CE0421B08F440E021E0628165
:104B500081810E9421250895EDE5F3E043812CE059
:104B6000420F08F44FEF21E0628181810E942125EC
:104B70000895EDE5F3E0628121E1621B08F460E055
:104B800021E0438181810E9421250895EDE5F3E034
:104B9000628121E1620F08F46FEF21E0438181819E
:104BA0000E9421250895EDE5F3E0818121E0438114
:104BB00062818C500E9421250895EDE5F3E081810A
:104BC00021E043816281845F0E94212508958091C4
:104BD000780380FD18C081FD14C082FD16C080914D
:104BE0007703882381F08C3380F427E0829FC00113
:104BF00011246CE370E00E94962C862F672B19F02D
:104C000005C083E0089581E0089587E008958091CC
:104C1000780380FD17C081FD17C082FD19C0809107
:104C20007603882399F08C3398F428E3829FC0019F
:104C300011246CE370E00E94962C862F672B49F4B8
:104C400081E008958EE008958CE1089588E008954C
:104C500088E30895282F35EB2303C001112497FF23
:104C600003C08058910902C080589F4F892F089532
:104C700060915D03669570E04BE050E08DE391E05C
:104C80000E94172E892B19F481E080938A030E94D9
:104C90007B219093840380938303089590915D0317
:104CA00090FF3EC09170811102C0926006C08B32AD
:104CB00010F0946502C0880F982B90935D036623D3
:104CC00091F020915D0330915E0340915F0350911C
:104CD000600360916103709162038091630390911E
:104CE00064030E94FC2360915D03669570E04BE0D5
:104CF00050E08DE391E00E94172E892B19F010925D
:104D00008A0302C00E94382681E08093860320E057
:104D10004091600360915F0380915E030E942125B2
:104D2000089561E00E944E26089580915D03869566
:104D3000815009F48AE261E00E944E260895809134
:104D40005D0386958F5F8B3208F081E061E00E9401
:104D50004E2608950E947B2120917E03211104C0DC
:104D600020917F03222321F090937C0380937B0387
:104D700020918003211104C020918103222321F07E
:104D800090937A0380937903E0916D03F0916E0321
:104D9000309731F00480F581E02D8DE793E009959F
:104DA0000895CF92DF92FF920F931F93CF93DF93DB
:104DB0006C010091EC0180919202082BC7E0D0E0D9
:104DC00010E0C8010C2E02C0959587950A94E2F771
:104DD00080FD04C02197A8F7F12C09C0FC2EB60174
:104DE0008C2F0E94290F0E94460F019799F38F2D57
:104DF000DF91CF911F910F91FF90DF90CF90089599
:104E0000CF93DF93EC010E94D126BE010E94290FAF
:104E10000E94460FDF91CF910895292F9E3078F59B
:104E2000863068F590E036E0239F800D911D1124B7
:104E3000682F677023E0969587952A95E1F7FC0126
:104E4000EE0FFF1FE80FF91FE557FC4F40E050E061
:104E500080E0219130E0062E02C0369527950A9415
:104E6000E2F721703327042E01C0220F0A94EAF7DB
:104E7000822B4F5F5F4F4330510559F7089580E013
:104E80000895292F9E3088F5863078F590E036E039
:104E9000239F800D911D1124282F277051E001C000
:104EA000550F2A95EAF723E0969587952A95E1F71D
:104EB000FC01EE0FFF1FE80FF91FE557FC4F20E044
:104EC00030E070E04081CB01022E02C096958795BC
:104ED0000A94E2F781708195842785238427819342
:104EE0002F5F3F4F2330310569F70895A0E2B0E00E
:104EF000ECE7F7E20C943D2B0E946E1C182F80917A
:104F0000CC028823A9F02FEF80E792E02150804067
:104F10009040E1F700C0000085E08983812F0E9466
:104F2000771B8A838EEF8B83CE0101960E941A1A1B
:104F30001093EC01A096E3E00C94592B21E030E0B3
:104F400001C0220F8A95EAF720958091EC01822317
:104F50000E947627089521E030E001C0220F8A9553
:104F6000EAF78091EC01822B0E94762708958093C6
:104F700092020895FC0124812223D9F0808191813D
:104F80000E94002792959F70963079F010F492500D
:104F900001C09A50923068F4803F69F018F4883E5E
:104FA00040F409C0843F29F406C0883E20F0813FC8
:104FB00011F080E0089581E0089580913401882304
:104FC00031F080919B0287FF02C08EE101C086E034
:104FD000E1E1F2E0DF011D928A95E9F780E090E0DF
:104FE0000E94322280E090E00E940D22109268031D
:104FF0000E94ED10EDE7F3E085E0DF011D928A9558
:10500000E9F71092760310927703109278030E94CA
:10501000AA260895882321F00E94DF100E94ED1037
:105020000895882339F090916803892B8093680351
:105030000E94ED100895882321F00E94E6100E943E
:10504000ED100895882339F090919E02892B80936A
:105050009E020E94ED100895662309F45CC08D3C09
:1050600021F40E940726819504C08E3C29F40E94F9
:10507000072680937F03C5C08F3C21F40E9407263A
:10508000819504C0803D29F40E94072680937E0309
:10509000B8C0893D19F40E94E72505C08A3D31F466
:1050A0000E94E725819580938003ABC08B3D21F45E
:1050B0000E94E725819504C08C3D29F40E94E725D4
:1050C000809381039EC09FE2980F983078F421E08E
:1050D00030E0A90102C0440F551F9A95E2F7CA01BA
:1050E00090917D03892B80937D038BC08D3D21F4AE
:1050F0008091780381600CC08E3D21F4809178030B
:10510000826006C08F3D09F07CC080917803846086
:105110008093780376C08D3C39F490917F0397FF9C
:1051200035C010927F0359C08E3C29F490917F03C3
:105130001916BCF32BC090917E038F3C29F497FF86
:1051400025C010927E0349C0803D19F41916CCF396
:105150001DC090918003893D29F41916BCF410926A
:1051600080033BC08A3D19F497FF10C0F8CF8B3DF8
:1051700039F49091810397FF09C0109281032DC0EB
:105180008C3D21F4909181031916BCF39FE2980F96
:10519000983080F421E030E0A90102C0440F551F8F
:1051A0009A95E2F7CA01809590917D0389238093B7
:1051B0007D0313C08D3D21F4809178038E7F0BC059
:1051C0008E3D21F4809178038D7F05C08F3D29F4B9
:1051D000809178038B7F8093780380917E03811187
:1051E00006C080917F03811102C0109276038091E6
:1051F0008003811106C080918103811102C0109249
:1052000077030E94AA260895882309F460C0823893
:1052100069F40E94572281FF5AC069E38FE092E04F
:105220000E94D8210E94ED1069E30EC0833899F4E2
:105230000E94572280FF4BC063E58FE092E00E94FE
:10524000D8210E94ED1063E58FE092E00E94B0212A
:105250000E94ED100895843869F40E94572282FF5D
:1052600036C067E48FE092E00E94D8210E94ED10E2
:1052700067E4EACF9CEF980F913A10F4682FE4CFDF
:1052800090E2980F983050F4877091E001C0990F28
:105290008A95EAF7892F0E94E610DACF9BE5980FEE
:1052A000933028F480E090E00E943222089598E53F
:1052B000980F9B3128F480E090E00E940D22089521
:1052C00093E3980F933118F460E00E942C2808951E
:1052D000CF93882309F4BDC0C82F8238B1F40E944F
:1052E000572281FDB6C069E38FE092E00E94D82189
:1052F0000E94ED102FEF87EE93E021508040904008
:10530000E1F700C0000069E317C08338E1F40E94B0
:10531000572280FD9EC063E58FE092E00E94D82175
:105320000E94ED102FEF81EE94E0215080409040DC
:10533000E1F700C0000063E58FE092E00E94B02139
:105340000E94ED1086C08438B1F40E94572282FD7D
:1053500080C067E48FE092E00E94D8210E94ED10A7
:105360002FEF81EE94E0215080409040E1F700C0A3
:10537000000067E4E1CF8CEF8C0F813AB8F58091A3
:1053800034018823E1F080919B0287FF18C0EC2F45
:10539000E695E695E695F0E0E15FFD4F8281282FE6
:1053A00030E04C2F477081E090E002C0880F991FD9
:1053B0004A95E2F782239323892B59F411C0E1E146
:1053C000F2E08191C81729F022E0E731F207C9F72E
:1053D00007C06C2F8FE092E00E94B0210E94ED1078
:1053E0006C2F8FE092E00E94D821AACF80E28C0F30
:1053F000883068F4C77081E090E001C0880FCA95DA
:10540000EAF790919E02892B80939E0299CFEBE55B
:10541000EC0FE33040F4F0E0EC5AFE4F808190E076
:105420000E94322216C0E8E5EC0FEB3150F4F0E0B8
:10543000EE0FFF1FE95AFE4F808191810E940D22DD
:1054400008C083E38C0F833120F461E08C2F0E942D
:105450002C28CF9108951F93CF93DF93182F893372
:1054600019F0C0E0D0E002C0C0E5D0E0812F0E947A
:105470006829209741F08FE99FE00197F1F700C07C
:1054800000002197F6CF812F0E940429DF91CF9150
:105490001F9108951092B9008CE08093B800089590
:1054A000A0E0B0E0E6E5FAE20C94352BB82EEB0173
:1054B0000E947B216C01C431D10558F0CF3F8FEFA2
:1054C000D80759F0CE0164E170E00E941A2B7B01ED
:1054D00007C0EE24E394F12C03C025E0E22EF12C6A
:1054E00084E8A82E94EA992E1092BC009092BC00F9
:1054F0000E947B218C018091BC0087FD07C0C80100
:105500000E946C21E816F906B0F729C08091B90015
:10551000887F883041F08091B900887F803119F010
:105520000FEF1FEF1EC0B092BB00A092BC000E9404
:105530007B218C018091BC0087FD07C0C8010E94BF
:105540006C21E816F906B0F70AC08091B900887F8F
:10555000883111F0803421F700E010E00EC00EEF2A
:105560001FEFCF3F8FEFD80709F4BECFC6010E94CF
:105570006C21C817D90708F0B7CFC801CDB7DEB77F
:10558000EBE00C94512B0F931F93CF93DF93EB0120
:105590008093BB0084E88093BC000E947B218C0137
:1055A0008091BC0087FD0DC0CF3F8FEFD807C1F3BE
:1055B000C8010E946C21C817D90790F78EEF9FEFA2
:1055C0000CC02091B900287F81E090E0283211F4CE
:1055D00080E090E0919581959109DF91CF911F91A5
:1055E0000F9108950F931F93CF93DF93EC0184E8FD
:1055F0008093BC000E947B218C018091BC0087FDC0
:105600000DC0CF3F8FEFD807C1F3C8010E946C21B6
:10561000C817D90790F78EEF9FEF03C08091BB00AA
:1056200090E0DF91CF911F910F91089584E98093CD
:10563000BC000895AA1BBB1B51E107C0AA1FBB1FDA
:10564000A617B70710F0A61BB70B881F991F5A950E
:10565000A9F780959095BC01CD0108952F923F92B6
:105660004F925F926F927F928F929F92AF92BF9272
:10567000CF92DF92EF92FF920F931F93CF93DF931E
:10568000CDB7DEB7CA1BDB0B0FB6F894DEBF0FBE7B
:10569000CDBF09942A88398848885F846E847D84C8
:1056A0008C849B84AA84B984C884DF80EE80FD80CA
:1056B0000C811B81AA81B981CE0FD11D0FB6F89440
:1056C000DEBF0FBECDBFED0108958F929F92AF92C6
:1056D000BF92CF92DF92EF92FF92CF93DF93EC01D4
:1056E000688179818A819B816115710581059105A8
:1056F00021F464E279ED8BE597E02DE133EF41E0B1
:1057000050E00E94192C49015A019B01AC01A7EA03
:10571000B1E40E94382C6B017C01ACEEB4EFA50122
:1057200094010E94462CDC01CB018C0D9D1DAE1D09
:10573000BF1DB7FF03C00197A109B04888839983B3
:10574000AA83BB839F77DF91CF91FF90EF90DF908B
:10575000CF90BF90AF909F908F9008950E94652B3F
:10576000089580E091E00E94652B0895A0E0B0E0EC
:105770008093000190930101A0930201B093030173
:105780000895F999FECF92BD81BDF89A992780B509
:105790000895A6E1B0E044E050E00C940B2CA8E1A1
:1057A000B0E042E050E00C940B2CDC01A40FB51FDC
:1057B0004150504048F0CB01840F951F2E910E941C
:1057C000E62B41505040D0F70895262FF999FECF8F
:1057D00092BD81BDF89A019700B4021639F01FBA44
:1057E00020BD0FB6F894FA9AF99A0FBE0895039661
:1057F000272F0E94E62B0E94E52B252F0E94E62BE7
:10580000242F0C94E62B0196272F0E94E62B0C9454
:10581000E52BDC01CB01FC01F999FECF06C0F2BDFE
:10582000E1BDF89A319600B40D9241505040B8F75E
:105830000895052E97FB1EF400940E94302C57FD0E
:1058400007D00E944B2C07FC03D04EF40C94302C54
:1058500050954095309521953F4F4F4F5F4F08959C
:1058600090958095709561957F4F8F4F9F4F0895CC
:105870000E946D2CA59F900DB49F900DA49F800D4C
:10588000911D11240895B7FF0C94382C0E94382CD8
:10589000821B930B0895A1E21A2EAA1BBB1BFD01CC
:1058A0000DC0AA1FBB1FEE1FFF1FA217B307E407FF
:1058B000F50720F0A21BB30BE40BF50B661F771F57
:1058C000881F991F1A9469F7609570958095909537
:1058D0009B01AC01BD01CF010895A29FB001B39F10
:1058E000C001A39F700D811D1124911DB29F700DE9
:1058F000811D1124911D0895991B79E004C0991F01
:10590000961708F0961B881F7A95C9F78095089519
:1059100087FB082E062687FD819567FD61950E940D
:105920007C2C0EF4919507FC8195089597FB072E2A
:1059300016F4009407D077FD09D00E941A2B07FCBB
:1059400005D03EF4909581959F4F0895709561958F
:105950007F4F0895EE0FFF1F0590F491E02D0994FD
:105960000E946D2C332312F48A1B9B0B0C94BA2CCF
:105970000E946D2CB7FF0895821B930B08950F931F
:10598000083090F0982F872F762F652F542F432FB4
:10599000322F22270850F4CF220F331F441F551FE8
:1059A000661F771F881F991F0A95B2F70F910895F8
:1059B00097FB10F8169400080F93083098F00850E1
:1059C000232F342F452F562F672F782F892F902D77
:1059D000F4CF059497958795779567955795479553
:1059E000379527950A95AAF70F9108950F931F935E
:1059F000CF93DF938230910510F482E090E0E09144
:105A0000AE03F091AF0320E030E0A0E0B0E03097CB
:105A100019F1408151810281138148175907C8F05B
:105A20008417950769F4109731F012960C9312972A
:105A300013961C9327C00093AE031093AF0322C0AC
:105A40002115310519F04217530718F49A01BD01C9
:105A5000EF01DF01F801DBCF21153105F9F0281B3B
:105A6000390B2430310580F48A819B8161157105E1
:105A700021F0FB019383828304C09093AF03809352
:105A8000AE03FE01329644C0FE01E20FF31F819384
:105A9000919322503109398328833AC02091AC0375
:105AA0003091AD03232B41F4209106013091070181
:105AB0003093AD032093AC03209104013091050194
:105AC0002115310541F42DB73EB7409108015091A1
:105AD0000901241B350BE091AC03F091AD03E217F3
:105AE000F307A0F42E1B3F0B2817390778F0AC0101
:105AF0004E5F5F4F2417350748F04E0F5F1F5093DE
:105B0000AD034093AC038193919302C0E0E0F0E0D9
:105B1000CF01DF91CF911F910F910895CF93DF9324
:105B2000009709F481C0FC01329713821282A09180
:105B3000AE03B091AF03109781F420813181820FC1
:105B4000931F2091AC033091AD032817390751F50D
:105B5000F093AD03E093AC0367C0ED0120E030E0CB
:105B6000CE17DF0740F44A815B819E014115510544
:105B7000F1F0EA01F5CFD383C28340815181840FD4
:105B8000951FC817D90759F488819981840F951FEB
:105B90000296918380838A819B81938382832115DE
:105BA000310529F4F093AF03E093AE033DC0E90162
:105BB000FB83EA8349915991C40FD51FEC17FD0768
:105BC00061F480819181840F951F0296E901998388
:105BD0008883828193819B838A83E0E0F0E0129640
:105BE0008D919C911397009719F0FD01DC01F7CF7F
:105BF0008D919C9111979D012E5F3F4F820F931FB6
:105C00002091AC033091AD032817390769F4309720
:105C100029F41092AF031092AE0302C013821282D5
:105C2000B093AD03A093AC03DF91CF910895FC0135
:105C30004150504030F001900616D1F73197CF0116
:105C40000895882799270895FB01DC0104C08D91F0
:105C50000190801921F441505040C8F7881B990BDE
:065C60000895F894FFCF47
:105C6600010000000000B0032000FF00991E32155D
:105C76002B1524150000000000002D1B601BBD1A0B
:105C860000000000000000000000111B491BA41AC0
:105C96000000000001010201C80001200001191ADC
:105CA6001B1C1D1E1F20212256476D72372F377071
:105CB60062797000818283E200E900EA00B500B6ED
:105CC60000B700CD008301CC008A01920194012126
:105CD60002230224022502260227022A02B300B466
:105CE600006F0070009F01CB019F02A00244224773
:105CF6006D1704F503AE0341036D048604A604BFC5
:105D06000400010202020206060609090909090938
:105D16000F0F0F0F0F0F1515151819191919191936
:0C5D2600191919192324252525252525E8
:00000001FF
